:020000040800F2
:2000000000200020B12A0008012B0008012B00080000000000000000000000000000000055
:20002000000000000000000000000000012B00080000000000000000012B00080324000829
:20004000012B0008012B000801260008012B0008012B00083129000841290008512900084B
:2000600000000000012B0008012B0008012B0008012B0008612D0008792D0008812D0008B6
:20008000992D0008012B0008012B0008B12D000800000000C92D0008E12D0008E50B000838
:2000A000FD0B0008012B0008012B0008012B0008012B0008012B00080000000002B47146BF
:2000C00049084900095C49008E4402BC7047C046002243088B4274D303098B425FD3030AF2
:2000E0008B4244D3030B8B4228D3030C8B420DD3FF22090212BA030C8B4202D312120902B2
:2001000065D0030B8B4219D300E0090AC30B8B4201D3CB03C01A5241830B8B4201D38B0389
:20012000C01A5241430B8B4201D34B03C01A5241030B8B4201D30B03C01A5241C30A8B42E4
:2001400001D3CB02C01A5241830A8B4201D38B02C01A5241430A8B4201D34B02C01A5241C1
:20016000030A8B4201D30B02C01A5241CDD2C3098B4201D3CB01C01A524183098B4201D3E5
:200180008B01C01A524143098B4201D34B01C01A524103098B4201D30B01C01A5241C308CF
:2001A0008B4201D3CB00C01A524183088B4201D38B00C01A524143088B4201D34B00C01A31
:2001C0005241411A00D20146524110467047FFE701B5002000F006F802BDC0460029F7D019
:2001E00076E770477047C04610B5064C2378002B07D1054B002B02D0044800E000BF01231D
:20020000237010BD8C000020000000006C330008044B10B5002B03D00349044800E000BFE2
:2002200010BDC04600000000900000206C33000810B50121152002F065FC0021152002F0DD
:20024000B5FC00211E2002F05DFC084C18222000192100F05DF900222000082100F08CF935
:200260002000034900F08DF910BDC046B0000020790200087047000073B52B4C2B48217814
:2002800000F0A0F80121152002F090FC0920FA21274E8900B3680093756801356843FFF75D
:2002A00017FF0022009B0193B36800930199009B99421DD20199009BEB1A5B18D218009BF8
:2002C00001939042F0D80021152002F06FFC01211E20184A02F038FE1125174B45431860BB
:2002E000164B174E9D4207D9C8239B0033600BE0019B00995B1AE1E764212800FFF7E8FE7A
:20030000104B9D4208D930603268C72A06DC13003C3BDBB2237073BD3C23E7E7CD23534338
:20032000DB127833F5E7C04600000020B000002010E000E080841E00AC0000207F380100DD
:20034000A8000020D3170000837D407D181A7047427D817D0300914204D90169885C013254
:200360005A75704701204042FBE7437D827D9A4202D90269D05C704701204042FBE7036DB9
:2003800010B51A00B0321268002A03D0002159779977904710BD000070B505000C00202901
:2003A00000D220242100A86902F030FF002802D0A8612C7770BD2100014802F029F9F9E7A3
:2003C0008433000813B56B46D971C37F0400002B17D0817F037F0131994201D9FFF7DCFF09
:2003E000A069002802D10123636016BD6B46DA79637FC254637F01200133DBB26377A3778B
:20040000F3E76B460122D91D243000F063FB43425841EAE770B5C37F04000E001500002BEE
:200420001AD0817F037F8918994201D9FFF7B4FFA069002804D1012305006360280070BD0A
:20044000637F2A00C018310002F026FE637F5B19DBB26377A377F1E792B2243000F03AFB05
:200460004342584140420540E8E7000000234360FA2301009B008360074B084A0833036024
:20048000074B78315B6A5B009B5A0B800300928B7A331A807047C046003400080C38000815
:2004A000E437000870B504000023B03440672360036143618361C3614B00441CDBB2050072
:2004C0003339E3774C426141AE3529700100AF310A70243001220849040000F04DFA2B78A9
:2004E000002B07D12000054900F012FB2000044900F004FB70BDC046A08601007F0300084E
:20050000BD05000810B50A003321FFF7CBFF10BD10B5132911D8164B49005B5E010078316A
:200520000B80132A16D8124B52009B5E02007A3200211380FFF7E6FF10BD1539CBB2092B54
:2005400005D80C4B8900CB5809495B00E5E701235B42E3E7153AD3B2092B05D8054B9200F0
:20056000D358034A5B00E0E701235B42DEE7C0460C380008E437000810B5C9B2FFF792FF1F
:2005800010BDB0300160704770B5037D05000C008B420AD2202900D220242100286902F034
:2005A00035FE002802D028612C7570BD2100024802F02EF8F9E7C04684330008F8B5046D71
:2005C00005002700B4373B68C66D002B1BD0627DA37D9A4217D331002000FFF7D5FF2369AC
:2005E000002B04D1CF210848490002F011F8290032002069683102F04FFD0023A6756375A6
:2006000030003B689847F8BD9C3300080300806910B5002803D000211A7F02F046FD10BD34
:20062000002110B50400417581750069884202D0227D02F03AFD002320006377A377FFF72A
:20064000E5FF10BD10B50248FFF710FF10BDC046B0000020134A030010B590421AD1C0226E
:20066000114B92015B6D134080225201934208D080229201934212D0002B05D101F004FDEF
:2006800001E00A4B186810BD0948E32101F0C0FF0020F8E7074A00209342F4D1EEE70648A5
:2006A000F1E7C04600540040001002402400002028340008005800400024F400F0B5A7B022
:2006C0001091109A9749D20003005058984205D1881840680190002800D01FE11C26924FCE
:2006E00058088B50C0191900FFF7F2FC109B8F4D5E437359040058081900C019FFF7E8FCC5
:20070000AD192B8BA9891193119A09908918A87EEA8AC31C0A920A9F6343EA893239D21B73
:20072000053AC91AFF3AE318D31A2A8A6043D2191892CA43D2171140DA43D2171340199140
:200740001290696878481A93FFF7C2FCA9681B907548FFF7BDFC129A63003233D2181592D8
:2007600062420892159AE31894460F93099BA44413931023624600271493113B1C900092B0
:200780000C970193249625950A99FBB28C46159A1793009B9B1A3A072292119A0B936244FF
:2007A00016921699099A511A009A52008A1A219200220392189A0B998A4200D992E02299B2
:2007C000039A0A4300211E920291199A8A4200D981E01A9A8A4200D27DE0149A1798824242
:2007E00079D00C9A01320C92072A00D996E0259A1E98528A1D92029A120410431F90169A55
:20080000009812180D920F9A24980492219A0E9200220792454A121823920498129A121886
:200820001D98904244D2049A323A920894423FD21F98079A0243209200980D9A0590121843
:200840000E988446002006901C9890421FD81B9890421CD32398059D808AA84217D8AC4253
:2008600015D20998161A00D56646139886420ED20698209D0002054310980195C000050044
:20088000284813964019019D4560179814900698089D013006906046AC46604484460598A3
:2008A000069DC01805908020D21840008542CBD10898079A8446013207920E9A0798624437
:2008C0000E920D9AD2180D92049AD2180492802252009042A1D1029AC91801320292102A74
:2008E00000D072E7802149038C460B9AD2180B92039A62440392802203995204914200D0D5
:2009000058E7089B01371B1B0893009B1B1900930F9B1B190F93102F00D035E7019827B06F
:20092000F0BDC0466801002000CA9A3B943400080E4A030010B5914212D90D4A914206D826
:200940000068FFF787FE0121FFF7B8FE10BD094A00209142FAD81868FFF77CFE0221F3E714
:200960000068FFF777FE0021EEE7C046A0860100801A060040420F00F0B587B0041E0191C0
:200980000292039374D00600484F543639000023F05E01F011FE23005633454905000020B9
:2009A000185E01F009FE0100002D61D000285FD0280001F00AFE2060002859D03D4B251D57
:2009C000984257D180223C4B9203D96B1143D963D96B114004910499D96A0A43DA62DA6AAC
:2009E00036490A40DA622300172258331A70344B1D60230056330020185E2D4901F0BAFD25
:200A00000023F05E390001F0B5FD2368019963602000FFF78DFF039B0022E360FF23A361D6
:200A2000029BA0602361230062618B331B782600591E8B41DB042362230000204533626212
:200A400058361A700221305600F05EF90020305600F084F9280000F07BFA002803D0194991
:200A6000194801F0D5FD0023E36589340233237007B0F0BD154B9842BBD180220E4BD20368
:200A8000D96B1143D963D96B114005910599D96A0A43DA62DA6A0E490A40DA62230018226F
:200AA00058331A70064B5D60A3E7C0464C360008103600080054004000100240FFFFDFFFE9
:200AC00080010020D50200002834000800580040FFFFBFFF030030B50120202A07D8002094
:200AE00084B2A24204D80020D2B288331A7030BD0D5C1C18683425700130F1E710B5002866
:200B000005D0002903D00166043000F04BFB10BD10B5002805D0002903D04166043000F0DD
:200B200041FB10BD836810B504009A4214D1230000220438853301290FD11A70436E9342E4
:200B400000D098472300843321001A788023200064319B0400F052FA10BDC26501221A7085
:200B60008023C16D5B0468314118200000F0AEFAF2E770B50600853633780400051F012BDD
:200B800005D1EB6D002B02D028002B6E98470223337000232000EB6500F004FB70BD836D23
:200BA000011F10B51F2B02DCCB6D0133CB65030085331B78DAB2012B06D1CB6D6833C918FB
:200BC00080235B0400F082FA10BD0023843003707047030010B586331B78002B01D100F0D8
:200BE000E1FA10BD044B10B51C68200000F0EEFA200000F0BFFE10BD80010020044B10B56E
:200C00005C68200000F0E2FA200000F0B3FE10BD8001002003000A4910B50868C318EFF3AD
:200C20000882934205D90C220120064B40421A6010BD054A054C121B9342F4D20B60F7E75D
:200C400004000020340300200020002000040000FEE7000016220120014B40421A60704798
:200C6000340300200120704770470000104B70B519680500002901D1012070BDFA208000A5
:200C8000FFF726FA0B4B01001868FFF721FA00F071F8041EF0D1032DEED8020001202900D8
:200CA000404200F031F8044B20001D60E5E7C04608000020240000200C0000208023084A4E
:200CC0005B00116810B50B4300201360FFF7CEFF041E03D1FFF7C8FF200010BD0124FBE730
:200CE00000200240034A0449136809685B1813607047C0463003002008000020014B186822
:200D00007047C0463003002030B5FF2503242A000440E400A24089012940D243A140C3B201
:200D200000280ADBC0240B4B80088000C018A40003591A401143015130BD0F200340083BEA
:200D400005489B089B001B18D86902401143D961F2E7C04600E100E000ED00E0002805DB4F
:200D60001F2318401E3B8340014A13607047C04600E100E08022431E5204012093420DD253
:200D8000C021074A07485360036A09061B021B0A0B43036200200723906013607047C04644
:200DA00010E000E000ED00E0704710B5FFF7FCFF10BD0000F8B50123411DCB77841DE27FE9
:200DC000022A03D00422C2631800F8BD0E2602681568B54315601568466C9D431560326856
:200DE000114D2A4032601C22AC46056C0F4E2A40934077683B437360C26C836C5A60036DE7
:200E0000002B06D065461A682A401A60436D826D5A600123E3770024CC77826B1300A2429E
:200E2000D2D090472300CFE7FFFEFFFF0000024070B5084D0400EB68184202D0E86001F0ED
:200E40006FFD2B69234203D020002C6101F06CFD70BDC0460018024003689A69920701D5E9
:200E600000229A6201229969114202D199690A439A61704730B5039C1204006822431A4344
:200E8000054B45688905640D890D1C43A5430A432A43426030BDC046FF63FF03042210B5DB
:200EA000436B174C0A40A34202D0164CA34214D100239A4200D0B83311220A40112A01D1B0
:200EC0007F32134312221140914201D14E32134301680A6813430B6010BD00239A4200D0D3
:200EE000B833CA0701D5F22213438A0701D5F4221343122211409142EAD10E32E7E7C046FC
:200F00005518000851170008002310B5CA0708D5030041331A7828231A401A33282A00D039
:200F2000B0338A0708D502002824413212782240A2420AD1442213434A0701D5B8221343E1
:200F400001680A689A430A6010BDF422F3E7704770B504000120002C3FD0250041352B7838
:200F6000DAB2002B05D12300403320001A70FFF7EEFF242301212B702368E0681A68A6685A
:200F80008A431A6061681A4A0A401A619968194A11409960012821D1802109023143996036
:200FA0005868154901435960D96800200A40DA60616922690A43A16909020A43DA60216A68
:200FC000E2690A431A60012219680A431A60202360642B7020634234207070BD842109028C
:200FE000314399600228DBD1802109015960D7E7FFFFFFF0FF7FFFFF00800002F0B50700F5
:2010000085B0029228220191039341373B78040001251340934208D1002902D0029B002B7C
:2010200006D1802301259B006364280005B0F0BD260005214036FFF767FF3378012B3DD022
:2010400035703B781E4D2A2B16D102212000FFF75BFF23681A6812040ED51A68E06B2A40C1
:201060001A60002808D0174B8363FFF7A3FE002802D0E06B836B984729233B7023002022A9
:2010800042331A7000232268636451680D4001995560616202996185618D21850399E162D1
:2010A000094961639169C90301D50821D161052120003370FFF7F2FE0025B6E70225B4E7D0
:2010C000FF7FFFFFD71900084D150008F0B5070085B0029228220191039341373B7804001C
:2010E00001251340934208D1002902D0029B002B06D1802301259B006364280005B0F0BD7A
:20110000260006214036FFF7FFFE3378012B3ED035703B78292B17D129002000FFF7F4FE6F
:2011200023681A6852040FD51A681A49A06B0A401A60002808D0184B8363FFF73BFE002814
:2011400002D0A06B836B98472A233B702300202242331A7000232268636451680F480140C4
:2011600051600199616202996185618D21850399E1620B4961639169C90301D40821D1615F
:20118000062120003370FFF789FE0025B5E70225B3E7C046FFBFFFFFD7190008FF7FFFFF30
:2011A0004D150008020010B5413211780223202907D126331370044B1C394363FFF76EFE34
:2011C0000023180010BDC0464D150008036810B599691A68436B002B00D0984710BD7047D7
:2011E0007047030070B500252022060042331D70013B1978040040361A7021290AD1112377
:20120000456303632039FFF77FFE20003570FFF7E6FF70BD1223456303630221FFF774FE59
:2012200020003570FFF7DCFFF3E7030070B5002542331D70013B1A780400292A0DD1013AB1
:201240001A70212301210363FFF75EFE2300403320001D70FFF7B9FC70BD1A782A2AFBD119
:20126000023A1A70222302210363FFF74DFE2300403320001D70FFF792FCEDE7F7B5FE272D
:20128000016804008D698E698B68CA68ED030192C268360CED0F3E40022A24D19B059A0DFE
:2012A0005B0F5E403000062318401E4210D1A36C0133A364A36C022B09D10633A064CB616B
:2012C00023004033187029002000FFF72BFCF7BD04212000FFF718FE2300002240331A7043
:2012E000019A3A40EFE70421FFF70EFE2300002240331A703200E6E7184B10B5C36200232B
:20130000020003630400202041321070537063634B0713D52368626A5B6A1370636A0133CB
:201320006362238D002B09D0013B2385638D013B9BB263850423626C134363640721200095
:20134000FFF7E2FD102223682000DA612300002240331A70FFF70DFC10BDC0460000FFFF8E
:20136000704770477047000070B5020005000026423241352B781670314A283BC262468516
:20138000426C04000A434264022B24D80321FFF7BBFD28232B702B4B2663636323688022D5
:2013A0001968D2010E00164011421FD01A682649A06B0A401A6000280CD0244B00228363F8
:2013C000230040331A70FFF7F5FC002802D0A06B836B984770BD0721FFF796FD2B78602B28
:2013E00001D020232B7000232363D6E718688021020009020A40084211D01A681449E06B0B
:201400000A401A600028E5D0104B8363230040331E70FFF7CFFC0028DCD0E06BD8E7230004
:2014200029784033602906D14039297020001A70FFF798FFCEE720001A70FFF7CAFBC9E725
:201440000000FFFF4D150008FFBFFFFFD7190008FF7FFFFF2022F8B5036804001D680F0002
:20146000DA610721FFF750FD802223681202596820000A435A605A6832490A405A60FFF766
:20148000EBFC01236A0438D5A36B002B03D01B685B689BB263857B0711D504239F43236843
:2014A000626A5B6A1370636A01336362238D002B05D0013B2385638D013B9BB26385638D6D
:2014C000002B03D00423626C13436364220000232500423223631370666C636341359E4227
:2014E00010D02000616CFFF73FFF2B78282B03D139002000FFF700FFF8BDED0B1D42CAD02D
:20150000E36BC2E72700E36A0F4A403793420BD02000FFF78AFE20230B4A2000E2622B70AB
:201520003E70FFF726FBE7E720232A7820002B703E70222A02D1FFF732FBDDE7FFF745FB8E
:20154000DAE7C04600E800FE0000FFFFF8B50700403716003A780400C36A0D000220012A62
:2015600023D0012209093A7011423ED0310911423BD0628D002A29D122004132117828291E
:2015800014D1802189048B4210D129002000FFF7B3FE0123AA0606D576091E4203D0290010
:2015A0002000FFF757FF00203870F8BD102110782268D1612928ECD136488342E9D02000A3
:2015C000FFF74AFC2000FFF730FEE2E710212268D1610422616C0A4362642F4A1342D8D158
:2015E0002000616CFFF7C0FED3E7012269071CD5B108114219D0628D002A0FD00422954321
:201600002268616A526A0A70626A01326262228D013A2285628D013A92B26285628D002A7D
:20162000B7D11C4A9342B4D0CCE70122290713D5F108114210D0230041331B782732134073
:20164000934203D12000FFF719FEA2E708222368DA6100233B709CE70122A90799D5710830
:20166000114200D195E7628D002A0DD0636A22681978013391626362638D013B9BB263859F
:20168000238D013B238584E7034A134200D080E798E7C0460000FFFFFFFFFFFE2022036847
:2016A00010B5DA615A680400274802405A60002222636263254AE262CA0605D51022DA61C3
:2016C0000423626C134363642000FFF7C5FB03212000FFF719FC22004132636C117860295D
:2016E00001D0002B04D02000616CFFF73DFE10BD1178212912D10139117022002100423207
:201700001078403113700B70402803D12000FFF727FEECE72000FFF762FDE8E71178222970
:20172000E5D1023911702200210042321078403113700B70402803D12000FFF712FED6E76A
:201740002000FFF74DFDD2E700E800FE0000FFFFF8B5050040352B780400C66A0220012B40
:2017600031D0012308092B70184250D0100918424DD0900BD20B84461043184243D0E76B3A
:20178000381E06D000201A4203D03B68586843425841A36B002B06D06246D20703D51B6862
:2017A0005B68002B01D001281ED1230041331A78282A09D180229204964205D12000FFF701
:2017C0009BFD00202870F8BD102219782368DA612929F6D11D498E42F3D02000FFF73CFB1C
:2017E0002000FFF722FDECE710222368DA610423626C13436364164B1E42E2D12000616C76
:20180000FFF7B2FDDDE710222368DA61D9E70123080710D5D00818420DD02300282241339F
:201820001B781340934203D12000FFF727FDC8E708222368E9E701238806C2D552091A42AB
:20184000BFD02000FFF706FEBBE7C0460000FFFFFFFFFFFE37B5050040352B78040002200F
:20186000012B17D0012308092B70184213D01009184210D0102223682000DA610423626CE8
:20188000122113436364FFF709FB2000FFF7E4FA002028703EBD0123080646D59009184217
:2018A00043D0402123681A688A431A60628D002A2FD05968638D8905890DFF2B1BD9FF2333
:2018C000238580235B040020228D0090D2B22000FFF7D0FA638D228D9B1A9BB263852300EF
:2018E00041331A7823681968222A0FD1802212020A431A60CCE7638DE26A23851C4B9A4253
:2019000001D0E36ADFE780239B04DCE78022D201EEE75B689B0103D42000FFF762FCB7E74C
:2019200040212000FFF720FDB2E70123480613D59009184210D0638D002BF1D123685A6823
:201940009201A5D4E16A0A4A9142E5D180225968D2010A435A609BE70123880600D497E790
:2019600052091A4200D193E72000FFF797FE8FE70000FFFF036870B59C6901211A68E50523
:2019800008D5D5090D4205D0456C2943416480214900D9610121650509D5D5090D4206D015
:2019A000456C0731294341648021C900D9610121A40509D5D2090A4206D00222416C0A43C5
:2019C000426480229200DA610B23416C194201D0FFF7CAFC70BD0023806A10B5826B93634D
:2019E000C26B9363030041331A78602A04D1403A1A70FFF7B7FC10BDFFF7EBF8FBE7000027
:201A000010B5114C1149236802000B4003432360802300209B009A420ED10D4B0D49186862
:201A200006235843FEF754FB8022431CD200616908001040114200D110BD002B01D0013B80
:201A4000F5E70320F8E7C04600700040FFF9FFFF2400002040420F00F0B5040085B0002821
:201A600023D00368DB0710D423689B075ED423681B0700D5C3E023685B0700D5F5E0E269DC
:201A8000002A00D07CE1002029E03822B04DAB681340EA68102B0AD1D243930709D12B6885
:201AA0009B03E1D56368002BDED1012017E0082BF5D0802263685202934212D12A681343BC
:201AC0002B60FFF71BF980270600BF022B683B42CAD1FFF713F9801B6428F7D9032005B087
:201AE000F0BDA021C9028B4208D180232968DB020B432B602B681A432A60E2E72A6895496A
:201B00000A402A602A6894490A402A60002BD8D1FFF7F4F880270600BF022B683B42A3D007
:201B2000FFF7ECF8801B6428F7D9D7E73823884DAA681340EA68102B28D103210A40022A61
:201B400026D12A68520502D5E268002AADD0696862698248120201400A436A60002B0DD102
:201B60002B687F4A1340226913432B602B687D4A9B045B0FDA4013007B4A13607B4B18683C
:201B8000FFF774F8002800D171E78EE7002BD8D0E368002B20D02B68714A80271340226911
:201BA000FF0013432B6080232A685B0013432B60FFF7A4F806002B683B4207D06A686369B7
:201BC00066491B020A4013436B6050E7FFF796F8801B0228EFD981E72B68654A80271340E2
:201BE0002B60FFF78BF80600FF002B683B4200D13DE7FFF783F8801B0228F6D96EE7382124
:201C0000534B9A681D000A40182A08D11B6E9B0700D430E7A369002B00D02CE745E7A2693B
:201C20000123002A10D02A6E022713432B66FFF765F806002B6E3B4200D01CE7FFF75EF840
:201C4000801B0228F6D949E72A6E02279A432A66FFF754F806002B6E3B4200D10BE7FFF77B
:201C60004DF8801B0228F6D938E73821384B9A681D000A40202A08D1DB6D9B0700D4FEE662
:201C8000A368002B00D0FAE60FE780220021DB6B52050091134208D1EB6B1343EB63EB6BF9
:201CA00013400393039B012300938027314E7F0033683B4215D0A368012B22D1EA6D13436D
:201CC000EB65FFF71BF802270600EB6D3B4238D0009B012B00D0D2E6EB6B274A1340EB63E8
:201CE000CDE633683B433360FFF708F8019033683B42E0D1FFF702F8019BC01A0228F6D9D6
:201D0000ECE6EA6D052B05D1013B1343EB65EA6D0123D4E701218A43EA65EA6D03318A43E6
:201D2000EA65002BCDD1FEF7E9FF02270600EB6D3B42CDD0FEF7E2FF104B801B9842F6D998
:201D4000CCE6FEF7DBFF0D4B801B9842BDD9C5E600100240FFFFFEFFFFFFFBFFFF80FFFF32
:201D6000FFC7FFFF0024F400240000200C000020FFFEFFFF00700040FFFFFFEF88130000E5
:201D80003820444B99681D000140102954D01B6841490B402B60022A37D1FEF7AFFF80273F
:201DA0000600BF042B683B4229D1616A236AEA680B433A4980260A401343E26AB604134333
:201DC000226B1343626B1343A26A12021343EB6080232A685B0413432B608023EA685B0572
:201DE0001343EB60FEF78AFF04002B68334200D049E6FEF783FF001B0228F6D96EE6FEF7E5
:201E00007DFF801B0228CDD968E60322EB6880269343EB60EB68224AB6041340EB60FEF742
:201E20006DFF04002B68334200D12CE6FEF766FF001B0228F6D951E6012A00D135E6032266
:201E4000DB68216A1A408A4200D02EE67022616A1A408A4200D028E6FE21A26AC9011940FB
:201E60001202914200D020E6F822E16A92031A408A4200D019E6E022216B12051A408A42EB
:201E800000D012E6626B5B0F5B07934200D1FAE50BE6C04600100240FFFFFFFE8C80C1113A
:201EA000FFFFFEEE38231E4A70B591681400194205D113681B489B045B0FD84070BD9168ED
:201EC0001940082927D091681940102917D1D368D168DB437F22E5684906490F2D0A01317E
:201EE00015409B0709D11048FEF7F2F8E1686843490F0131FEF7ECF8E0E70A48F4E7916896
:201F00001940202909D0926800201340182BD5D1FA20C001D2E70448D0E780200002CDE703
:201F2000001002400024F40000127A00F7B505000E00002801D10120FEBD07274A4C2368C7
:201F40003B408B422AD329688B073BD4CB0748D4072723683B40B3420AD92368BB43334311
:201F60002360FEF7CBFE019023683B40B3426BD12B683E4C5B076FD4FFF794FFA3683C4A7C
:201F80001B051B0F9B009B581F221340D840394B1860394B1868FEF769FECDE72368BB4324
:201FA0000B432360FEF7AAFE019023683B40B342C9D0FEF7A3FE019BC01A304B9842F4D960
:201FC0000320B9E7294A4B0704D5E0239068DB010343936093682A480340A8680343936097
:201FE000B4E76A68214F012A19D13B689B03A2D50721BB688B431343BB60FEF77FFE0190AA
:020000040800F2
:202000003823BA681A406B68DB009A42A0D0FEF775FE019BC01A194B9842F1D9D0E7022A26
:2020200003D13B689B01E3D485E7002A03D13B685B05DDD47FE70223032A03D1396E19422A
:20204000D6D178E7F96DFAE7FEF758FE019BC01A0A4B984288D9B3E7A3680A4A1340EA6844
:202060001343A36088E7C046002002400010024098350008240000200C00002088130000FE
:20208000FFF0FFFFFF8FFFFF064B074A9B685B045B0F9B009B581F221340044A1068D84059
:2020A0007047C04600100240D835000824000020036810B59A690400D20408D50122196D25
:2020C000114204D0D96D0A43DA6500F08BFA23689A69920409D50222196D114205D0D96D78
:2020E00020000A43DA6500F004F801232934237010BD7047704770470222036810B519696C
:20210000040011420ED0D96811420BD0053A1A61043202779B699B0700D186E000F0BEFE29
:2021200000232377042223681969114211D0D96811420ED0093A1A61073222779A69C02393
:202140009B0020001A4200D175E000F0A7FE0023237708222368196911420ED0D9681142F4
:202160000BD0113A1A610D322277DB6920009B0767D000F093FE002323771022236819692C
:20218000114210D0D96811420DD0213A1A6119322277DA69C0239B0020001A4257D000F08D
:2021A0007DFE00232377012223681969114207D0D968114204D0033A20001A6100F03CFE23
:2021C000802223681969114208D0D968114205D0023AFF3A20001A6100F0A6F823681A6910
:2021E000D20507D5DA68120604D51C4A20001A6100F09BF8402223681969114207D0D9689B
:20220000114204D0813A20001A61FFF774FF202223681969114207D0D968114204D0413A7C
:2022200020001A6100F07FF810BD00F033FE2000FFF760FF74E700F02DFE2000FFF75AFF54
:2022400085E700F027FE2000FFF754FF93E700F021FE2000FFF74EFFA3E7C046FFFEFFFF1D
:202260001D4A10B50368904206D08024E405A04202D01A4CA0420CD17024A3434C68234325
:2022800090420FD08024E405A0420BD0134CA04208D0134CA04205D0124CA04202D0124CA4
:2022A000A04203D1114C2340CC6823438024A3434C69234303608B68C3620B6883629042C4
:2022C00005D0084B984202D0074B984201D10B6903630123436110BD002C0140000400400C
:2022E000002000400044014000480140FFFCFFFF70B504000120002C14D025003D352B78E3
:20230000DAB2002B05D123003C3320001A7000F095FA02232B702068211DFFF7A1FF012335
:2023200000202B7070BD7047704770477FB5002304280FD81B4B5A6BFDF7C0FE030F1821FE
:202340002A0001210A435A635B6B0B400193019BA023DB05180007B000BD02210A435A638A
:202360005B6B0B400293029B0F4BF3E704210A435A635B6B0B400393039B0C4BEAE7082121
:202380000A435A635B6B0B400493049B084BE1E720210A435A635B6B0B400593059B054BED
:2023A000D8E7C046001002400004005000080050000C00500014005073B50E4E3368FEF786
:2023C0009DFC7568B3680135EB1A019333680400DB0305D5FEF792FC0400B368EB1A01930B
:2023E000FA260198B60029007043FDF771FE7443001976BD10E000E010B5FEF77FFC10BD5A
:20240000704710B5FEF76EFCFEF7CFFCFFF7F8FF10BD10B5FEF752FC00F006FB10BD431C42
:2024200004D100207047834205D00C3100228B5E5A1CF8D1F5E70120F4E700000F23F0B520
:20244000072587B082B204091C4003920340454A9B009F5802910D40431C17D14821424869
:2024600000F0D6F83E002000FFF760FF03237E437343D94382680400134301918360032D49
:2024800041D82800FDF71AFE3333233383B2093B032BE7D80126354A116C31431164136C42
:2024A00033400593059B324B0B2809D00C280BD0082219680A2800D110220A431A60D1E77A
:2024C00008211A688A43F9E710211A68FAE7029B5904039B490E1B070BD50F203B0A5B430D
:2024E0005B4358434B43626A8243134363622B000EE032000F20724350435143236A8343C0
:202500000B432362F3E78D21174800F081F80023734322680199013D0A4013432360012D0C
:2025200005D8029B1B070DD563683B436360029B9906890F012908D002290DD0E668019B49
:202540001E4006E06368BB43F0E7E368019A13401E43E66007B0F0BDE368019A76001340A4
:20256000F6E7C04658350008E8340008001002400000014010B5431C07D110BD834203D1CA
:202580008968FFF75BFFF8E70C3100228B5E5A1CF4D1B921014800F03BF8EEE7E834000859
:2025A00000228B5E5A1C01D1002002E0834201D1486870470C31F3E7030010B500205A1C53
:2025C00002D01800FFF7ECFF10BD030008008B4204D0002B02D0002901D1180070470020D0
:2025E000FCE70000044B10B51B68002B02D0034A1068984710BDC04688010020B80100206B
:2026000010B50248FFF754FD10BDC0468C010020FEE700008022024B12059A607047C04642
:2026200000ED00E00438704710B50368294A86B0934217D1802428492401086C20430864C7
:202640000A6C22400092009A244A934235D18020214AC002116C01431164136C03400593D0
:20266000059B2AE08022D205934213D01C4A93421AD01C4A934222D01B4A9342E4D180209E
:20268000154A8002116C01431164136C03400493049B12E001241049C86B2043C863CA6BC5
:2026A00022400192019ACFE702200B4AD16B0143D163D36B03400293029B06B010BD8020D3
:2026C000054A0002116C01431164136C03400393039BF2E7002C014000100240004801405C
:2026E0000004004000200040004401400368194A93420BD1184919480A6C02400A64184AE8
:2027000093421FD1144A1749136C1FE08022D20593420CD0144A93420FD0144A934212D067
:20272000134A9342EBD10C4A1249136C0EE001200949CA6B8243CA63E1E70221064AD36B7A
:202740008B43D3637047044A0B49136C0B401364F8E7C046002C014000100240FFF7FFFF43
:2027600000480140FFFFFBFF000400400020004000440140FFFFFDFFFF7FFFFF010010B573
:20278000431C14D00F4B0D20994212D012D80E4B033099420DD00D4B0330994209D08023A2
:2027A0000438DB05994204D00948FFF731FF0E20404210BD074B15209942FAD0064B0130AC
:2027C000F0E7C046002C01400004004000200040F83500080044014000480140010010B502
:2027E000431C14D00F4B0E20994212D012D80E4B023099420DD00D4B0330994209D0802342
:202800000438DB05994204D00948FFF701FF0E20404210BD074B15209942FAD0064B01307B
:20282000F0E7C046002C01400004004000200040F8350008004401400048014070B504003E
:20284000FFF7F2FE2068FFF799FF626C216CFEF75BFA2068FFF792FFFEF780FA2068FFF7DB
:20286000BDFF06002068FFF789FF86420BD02068FFF7B4FF626C216CFEF746FA2068FFF7AE
:20288000ADFFFEF76BFA70BDF8B5134F05003900FFF792FE00F0C6F9104E8400A359002B7A
:2028A0000DD139002800FFF787FE0700A82000F043FB0500390000F0FDF9A3591D60335938
:2028C0001C68002C06D0200000F0D6F9A821200000F036FBF8BDC04688360008FC020020EA
:2028E000836810B50400002B02D0032201009847200010BD002310B5012803D001334008D5
:20290000DBB2F9E714225343044A181D80188168002902D0D2181369984710BDBC01002090
:2029200010B5FFF7E7FF10BD10B5FFF7E3FF10BD10B50120FEF77CFA0220FEF779FA10BD17
:2029400010B50420FEF774FA0820FEF771FA10BD70B50C241025A8B2013CFEF769FA6D00F0
:20296000002CF8D170BD0000274B10B505211C001800002219701975283401312170083014
:202980001C00C26718003C3421708C30013101701800983002601800A03001701800AC30EB
:2029A00002601800B43001701800C03002601800C83001701C0018005034D43002602170AE
:2029C00018001C00DC3064340170217018001C00E83078340260217018001C00F030FF34AB
:2029E00001706171617618009624FC306400DA601A625A639A64DA651A6702604261826241
:202A00001955C26310BDC046BC01002010B5044C143C201DFFF764FF024B9C42F8D110BDB7
:202A2000FC020020BC01002000B593B03822002104A800F03AFB10220021684600F035FB36
:202A400080208000FEF7DCFF022304930B930C9306330E9380239B020F93802380229B04ED
:202A60005200109380234021079200229B0504A8089209910D921193FEF7EEFF002803D002
:202A80006F210A48FFF7C4FD07230221009300236846019102930393FFF748FA002803D0FC
:202AA00079210248FFF7B4FD13B000BD783700080D488546002103E00C4B5B58435004315E
:202AC0000B480C4B42189A42F6D30B4A02E0002313600432094B9A42F9D3FFF79BFD00F0D0
:202AE000A3FA00F01FFAFEE7002000207C390008000000208C0000208C000020440300206F
:202B0000FEE70000F7B50E00132827D8224B4000C45E631C30D00F2325091D401F4F234000
:202B20000193AD00EB59019AD340DB070ED520001B49FFF774FC002802D02000FFF7A4FE01
:202B40000123019A93407A599A437A51052E1ED83000FDF7B3FA0D181214161A1538092875
:202B60000AD8104B8000C3580B4A5B009C5ED0E700212000FFF762FCF7BD1021F9E7202181
:202B8000F7E70321F5E70121F3E70921F1E749210548FFF73DFDEFE70C3800081403002019
:202BA00088360008E437000834380008132813D8114B4000C35E1A060020120F042A02D86C
:202BC0000E48920010580F2213400D4A9B009B5800290ED0836170471538092806D8094BEA
:202BE0008000C358044A5B009B5EE4E701235B42E1E78362EFE7C0460C3800081000002007
:202C000058350008E4370008836810B50400002B05D00322010098470023A360E3602000BA
:202C200010BD00000E4A0300904215D08022D205904213D00B4A022093420CD00A4A0130DA
:202C4000934208D0094A0130934204D00848094A934200D1052070470020F8E70120F6E778
:202C6000002C0140000400400020004000440140FFFF00000048014070B504000069FFF7AF
:202C8000D1FF050020001030FFF730FD0023084AAD00AB5026002500E360A8355836B542CF
:202CA00004D0103D2800FFF71BFEF8E7200070BDFC0200200023F7B5021D03660367D36777
:202CC000843204009360080093610E00FFF7AAFF204F0500B84203D12F211F48FFF798FC1B
:202CE00023001E4AAD000C33AB50220000232C32266113702600203223636363A363E363A5
:202D000023646364A364137053700322103663653000E4602265FFF787FC23002500A8334E
:202D2000583501932800FFF76FFF019B10359D42F8D1002323606360A3606361A3612362A4
:202D4000636280333000E761A362FFF7D1FA2000FEBDC046FFFF00009B380008FC020020E5
:202D6000044B10B51868002802D00430FFF7C4F910BDC046FC02002010B5FFF7F1FF10BD75
:202D8000044B10B55868002802D00430FFF7B4F910BDC046FC020020044B10B59868002861
:202DA00002D00430FFF7A8F910BDC046FC020020044B10B5D868002802D00430FFF79CF978
:202DC00010BDC046FC020020044B10B51869002802D00430FFF790F910BDC046FC020020CF
:202DE000044B10B55869002802D00430FFF784F910BDC046FC020020836810B5002B01D1BF
:202E000000F060FAC368984710BD000010B5041E03D107490748FFF7FBFB2000FFF702FC37
:202E20000068036E002B02D05830FFF7E5FF10BD260400009B38000810B5FFF7E7FF10BD1A
:202E400070B5051E03D111491148FFF7E1FB287F0138072812D8FDF731F91604111211115B
:202E6000111402242800FFF7DDFB24010068583400198368002B01D0FFF7BEFF70BD0324F1
:202E8000F0E70424EEE70124ECE7C046390400009B38000810B5FFF7D3FF10BD10B5FFF733
:202EA000CFFF10BD10B5040000F0B4F8E06023682000DB689847002808DA00F0ABF8E3681D
:202EC000C01AA3689842F2D30120404210BDF8B506000D0017000024BC4207D03000FFF708
:202EE000E1FF002802DB28550134F5E72000F8BDF7B506000F001D001C1E01920CD00024DF
:202F00003000FFF7CFFF002806DBB84204D0019B18550134A542F3D12000FEBD10B500F06D
:202F200075F810BD10B500E000BFFDF781F9FDF7A1F900F077F8FAE710B500F099F810BDA4
:202F400010B500F09FF810BDF7B50D00009213280DD82B4B4000C35E0F2219000124114056
:202F60001B098C401340042B14D9002615E01538092824D8234B8000C2580F200124204E93
:202F80005200915B935F01401B098C4000260340042B02D81C4A9B009E58002D00D0250045
:202FA00000F03CF8070033692340AB420AD100F035F8009BC01B9842F5D90020FEBD802465
:202FC0002402D2E733692340AB4206D000F026F8009BC01B9842F5D9EFE700F01FF80190B6
:202FE00033692340AB4206D100F018F8009BC01B9842F5D9E1E700F011F8019BC01ADDE7F5
:203000000C380008E43700081000002010B5FFF700FA10BD10B5FFF7EFF910BD10B5FFF764
:20302000CBF910BD7047000070B500260C4D0D4C641BA410A64209D1002600F097F90A4D59
:203040000A4C641BA410A64205D170BDB300EB5898470136EEE7B300EB5898470136F2E736
:203060006439000864390008643900087439000810B5034B0100186800F06AF810BDC046F3
:203080002800002010B5034B0100186800F016F810BDC04628000020002310B59A4200D1A6
:2030A00010BDCC5CC4540133F8E703008218934200D1704719700133F9E7000070B505002F
:2030C000002910D00C1F2368002B00DAE418280000F0BAF81D4A1368002B05D1636014604C
:2030E000280000F0B9F870BDA34208D9216860188342F3D118685B6841182160EEE71A007E
:203100005B68002B01D0A342F9D911685018A0420BD120680918501811608342E0D1186822
:203120005B68411811605360DAE7A04202D90C232B60D5E721686018834203D118685B687E
:203140004118216063605460CAE7C04628030020F8B50323CD1C9D43083506000C2D1FD213
:203160000C25A9421ED8300000F06EF825490A681400002C1AD1244F3B68002B04D1210075
:20318000300000F04DF838602900300000F048F8431C2BD10C233000336000F05DF803E034
:2031A000002DDEDA0C2333600020F8BD23685B1B19D40B2B03D92360E418256003E06368E1
:2031C000A2420ED10B60300000F046F8200007220B30231D9043C21A9842E6D01B1AA35038
:2031E000E3E75360EFE722006468C2E70323C41C9C43A042E1D0211A300000F011F8431CAA
:20320000DBD1C7E7280300202C03002010B5034B0A000100186800F027F810BD28000020F8
:20322000002370B5064D040008002B60FDF7F2FC431C03D12B68002B00D0236070BDC04603
:20324000340300207047704710B50248FFF7FAFF10BDC0463C03002010B50248FFF7F3FF82
:2032600010BDC0463C030020F8B507000D001600002905D11100FFF76BFF04002000F8BDFC
:20328000002A03D1FFF71AFF3400F7E700F012F82C00B042F2D231003800FFF759FF041E5A
:2032A000ECD029003200FFF7F7FE29003800FFF705FFE3E70B1F1B68181F002B01DA0B589A
:2032C000C018704710B500F000F8062010B500F02DF80120FDF7BCFC70B504000D001F2967
:2032E00004D9162303600120404270BD436C002B04D08A009B181A68002A08D1200000F005
:2033000031F82A000100200000F01AF8EDE70020012AEAD0511C03D1162301302360E4E765
:20332000002428001C6090472000DEE710B5034B01001868FFF7D0FF10BDC0462800002095
:20334000002370B5064D0400080011002B60FDF781FC431C03D12B68002B00D0236070BD48
:203360003403002010B5FDF77DFC10BDF8B5C046F8BC08BC9E467047F8B5C046F8BC08BC06
:203380009E4670474E6F20656E6F756768206D656D6F72792120282569290A00433A5C551E
:2033A000736572735C673530305C446F63756D656E74735C41726475696E6F446174615CE6
:2033C0007061636B616765735C53544D33325C68617264776172655C73746D33325C312E7F
:2033E000392E305C6C69627261726965735C576972655C7372635C576972652E6370700022
:203400000000000000000000C50300081504000849030008510300086B0300082106000866
:20342000CF2E0008F12E0008433A5C55736572735C673530305C446F63756D656E74735CB3
:2034400041726475696E6F446174615C7061636B616765735C53544D33325C68617264775E
:203460006172655C73746D33325C312E392E305C6C69627261726965735C576972655C73D2
:2034800072635C7574696C6974795C7477692E6300000000A086010080380100C0D4010031
:2034A00000007A0DFA005C12A00F800214000000801A060000E20400005307000000840371
:2034C000640014055802FA006400000040420F0000350C00804F12000000C2013200F4011A
:2034E00004013C0064000000433A5C55736572735C673530305C446F63756D656E74735C7A
:2035000041726475696E6F446174615C7061636B616765735C53544D33325C68617264779D
:203520006172655C73746D33325C312E392E305C6C69627261726965735C53726357726125
:20354000707065725C7372635C73746D33325C70696E6D61702E6300010000000200000086
:2035600004000000080000001000000020000000400000008000000000010000000200004C
:2035800000040000000800000010000000200000004000000080000000000000000000002F
:2035A000000000000000000000000000000000000000000000000000010000000200000008
:2035C0000300000004000000060000000700000008000000090000000000000000000000C6
:2035E00000000000000000000100000002000000030000000400000054494D3A20556E6B4F
:203600006E6F776E2074696D6572204952516E0009000000005400400A0600000B00000075
:20362000005800400A06000016000000005400400A06000018000000005400400A0600006C
:20364000FFFF000000000000000000000A000000005400400A0600000C000000005800401A
:203660000A06000017000000005400400A06000019000000005400400A060000FFFF0000C4
:20368000000000000000000000000000000000401282000001000000000000401202010000
:2036A00002000000000000401282010008000000002C01401282000009000000002C0140B4
:2036C000120201000A000000002C0140128201000B000000002C0140120202000F0000002C
:2036E000000000401282000010000000002C0140120211001000000000040040128101006C
:2037000011000000002C0140128211001100000000040040120102001100000000200040AB
:203720001280000015000000000400401201010016000000002C014012810100160000005D
:203740000044014012821000170000000048014012821000180000000044014012820000CB
:20376000190000000048014012820000FFFF00000000000000000000433A5C55736572732A
:203780005C673530305C446F63756D656E74735C41726475696E6F446174615C7061636B20
:2037A000616765735C53544D33325C68617264776172655C73746D33325C312E392E305C47
:2037C00076617269616E74735C444953434F5F47303331365C76617269616E742E63707081
:2037E0000000000000000000010000000200000006000000070000000800000009000000A8
:203800000B0000000C0000000F000000000001000200080009000A000B000C000D000E0032
:203820000F0010001100150016001700180019002E004200433A5C55736572735C67353062
:20384000305C446F63756D656E74735C41726475696E6F446174615C7061636B61676573E7
:203860005C53544D33325C68617264776172655C73746D33325C312E392E305C636F72657D
:20388000735C61726475696E6F5C776972696E675F6469676974616C2E6300433A5C55730C
:2038A0006572735C673530305C446F63756D656E74735C41726475696E6F446174615C70E4
:2038C00061636B616765735C53544D33325C68617264776172655C73746D33325C312E39B1
:2038E0002E305C636F7265735C61726475696E6F5C486172647761726554696D65722E6388
:203900007070000000000000000000000000000000000000000000000000000000000000C7
:20392000000000000000000000000000000000000000000000000000000000000000000087
:20394000000000000000000000000000000000000000000000000000000000000000000067
:20396000000000001D2F0008110200084506000869290008E90100080D2A0008C8000000F2
:20398000480300200100000004000000000000500004005000080050000C005000140050FB
:2039A0000024F4002C00002000000000243900084439000804390008000000000000000074
:2039C0000000000000000000000000000000000000000000000000000000000000000000E7
:2039E0000000000000000000000000000000000000000000000000000000000000000000C7
:203A00000000000000000000FFFFFFFFFFFFFFFFFFFFFFFFFFFFFFFFFFFFFFFFFFFFFFFFBE
:203A2000FFFFFFFFFFFFFFFFFFFFFFFFFFFFFFFFFFFFFFFFFFFFFFFFFFFFFFFFFFFFFFFFA6
:203A4000FFFFFFFFFFFFFFFFFFFFFFFFFFFFFFFFFFFFFFFFFFFFFFFFFFFFFFFFFFFFFFFF86
:203A6000FFFFFFFFFFFFFFFFFFFFFFFFFFFFFFFFFFFFFFFFFFFFFFFFFFFFFFFFFFFFFFFF66
:203A8000FFFFFFFFFFFFFFFFFFFFFFFFFFFFFFFFFFFFFFFFFFFFFFFFFFFFFFFFFFFFFFFF46
:00000001FF
